:020000040000FA
:10000000A8260020F90200000103000003030000FD
:1000100005030000070300000903000000000000C2
:100020000000000000000000000000000B030000C2
:100030000D030000000000000F030000110300008A
:100040001303000013030000D9070000130300008E
:100050001303000013030000A103000013030000BA
:100060001303000013030000130300001303000038
:100070001303000013030000130300001303000028
:1000800013030000130300004105000013030000E8
:100090001303000013030000130300001303000008
:1000A00013030000130300001303000013030000F8
:1000B0001303000013030000000000000000000014
:1000C00013030000130300001303000013030000D8
:1000D00013030000130300001303000013030000C8
:1000E00013030000130300001303000000000000CE
:1000F00000000000130300000000000013030000D4
:1001000000000000000000000000000000000000EF
:1001100000000000000000000000000000000000DF
:1001200000000000000000000000000000000000CF
:1001300000000000000000000000000000000000BF
:1001400000000000000000000000000000000000AF
:10015000000000000000000000000000000000009F
:10016000000000000000000000000000000000008F
:10017000000000000000000000000000000000007F
:10018000000000000000000000000000000000006F
:10019000000000000000000000000000000000005F
:1001A000000000000000000000000000000000004F
:1001B000000000000000000000000000000000003F
:1001C000000000000000000000000000000000002F
:1001D000000000000000000000000000000000001F
:1001E000000000000000000000000000000000000F
:1001F00000000000000000000000000000000000FF
:10020000DFF80CD000F0BAF800480047450E0000B7
:10021000A826002030B4044654E8000F0D4644E8F8
:100220000053002BF8D1156030BC704730B4044641
:1002300054E8000F40EA010544E80053002BF7D1D1
:10024000156030BC704730B4044654E8000F00EA33
:10025000010544E80053002BF7D1156030BC70470E
:1002600030B4044654E8000F80EA010544E8005326
:10027000002BF7D1156030BC704730B4044654E809
:10028000000F00EB010544E80053002BF7D1156087
:1002900030BC704730B4044654E8000FA0EB0105B1
:1002A00044E80053002BF7D1156030BC704770B4A0
:1002B00004464FF0000054E8006F0D68AE4207BFDF
:1002C00044E80023012044E800630E60002B1CBFBB
:1002D0000020F0E770BC704730B4044654E8000FCB
:1002E00088422CBF451A054644E80053002BF5D13F
:1002F000156030BC7047000006488047064800473C
:10030000FEE7FEE7FEE7FEE7FEE7FEE7FEE7FEE7C5
:10031000FEE7FEE7FD05000001020000004870470F
:10032000702C000040EA01039B0703D009E008C9D4
:10033000121F08C0042AFAD203E011F8013B00F8AA
:10034000013B521EF9D27047D2B201E000F8012BF6
:10035000491EFBD270470022F6E710B513460A4645
:1003600004461946FFF7F0FF204610BD421C10F866
:10037000011B0029FBD1801A70470000064C074D75
:1003800006E0E06840F0010394E807009847103465
:10039000AC42F6D3FFF738FF182D0000382D0000CF
:1003A0002DE9F04F00258BB0DFF88C81A94606952A
:1003B0004FF4807601242F460795304601F0E0F88F
:1003C00038B1D8F80403204203D0304601F0CEF80B
:1003D0002543361D64007F1CB6B2082FEDD34FF4C1
:1003E000BE74204601F0CCF848B1204601F0BEF8BA
:1003F00045F0004506AA0221002001F0A1F84F4E69
:1004000015F0FF0F15D0012700242F420DD008EB67
:100410008401D1F81005D1F81015C0F3052056F865
:100420002420C1F3014102B190477F00641C082CD5
:10043000EBD3002D46DA0020CDF82090411E0DF1BF
:10044000180A04AC0DF1040BCDF8249044F82010E8
:10045000401C0228FAD396F85470002578B227F091
:10046000C008401C2ED004A9404600F011FE002810
:1004700028D04FEA9719404600F02AFB56F8207022
:100480001FB1B9F1030F03D006E0B9F1030F19D181
:1004900008A9404600F004FE02A8CDF8088000F04C
:1004A000FBFF029900EB8100D0F8000706A9C0F31A
:1004B00001400290404600F0EBFD0028029804D075
:1004C000022804D00BB0BDE8F08F0328FAD1B9F1AF
:1004D000030F07D10298022828D00221404600F0DD
:1004E000B9FF012517B149464046B847002DE9D06C
:1004F00001AA0221002001F023F8002052465946AB
:1005000052F8207051F82030BB4211D0002008ABC7
:1005100051F8207042F8207053F8207044F8207091
:10052000401C0228F4D3002D95D1CBE70321D5E759
:10053000401C0228E4D3C5E700600040D40000203E
:100540002DE9F8432A48DFF8A4804FF4807201684F
:10055000284E002589B1D8F8041311F0010F0CD0F2
:10056000056000680090244862F30F040068726818
:1005700060F317443946204690471D484FF4827176
:10058000001D0268BAB1D8F8042312F0020F12D08D
:10059000056000680090184861F30F040C30006893
:1005A00060F31F4414483C300068726860F30F0722
:1005B0003946204690470E484FF484720830414631
:1005C0000368002B10D0D1F8041311F0040F0BD0E6
:1005D000056000680090204662F30F00726801B069
:1005E0003946BDE8F0431047BDE8F88300200140DC
:1005F00000210140340000200C25014030B54FF0AF
:10060000805000228300D0F83011C3F80C21C3F8C9
:100610001021624B1A60624B1B68624C2360604B76
:100620001B1D1B68241D23605D4B08331B68241DA4
:1006300023605B4B0C331B68241D2360584B103325
:100640001B68241D2360564B14331B68241D236034
:10065000534B18331B68534C20342360504B1C33CE
:100660001B68241D23604E4B20331B68241D236010
:100670004B4B24331B68241D2360494B28331B68D4
:10068000241D2360464B2C331B68241D2360444BE0
:1006900030331B68434C40342360414B34331B6878
:1006A000241D23603E4B38331B68241D23603C4BC4
:1006B0003C331B68241D2360394B40331B68241DC9
:1006C00023600124082902D1D0F8343113B108295C
:1006D00004D006E0354B3449196005E0D0F83431D8
:1006E00013B1082904D006E0314BFB21196005E065
:1006F000D0F8343113B1082908D00EE090F8583200
:100700002C48016863F30301016002E0D0F8343142
:100710001BB929494FF40070086028480168C907CF
:1007200002D06FF0010101602548016841F47001B9
:100730000160BFF34F8FBFF36F8F4FF01021D1F8DF
:100740000002002803DBD1F80402002822DA1D4B46
:100750001C601D480468002CFCD01224C1F8004223
:100760000568002DFCD0C1F8044201680029FCD0C6
:100770001A6001680029FCD0BFF34F8F10487C3805
:100780000168124A01F4E06111430160BFF34F8F29
:1007900000BFFDE70F490E48086030BD3805004036
:1007A0000404001020C50040488103008C5600401E
:1007B00018F50040E40E004040960240000400405E
:1007C00088ED00E004E5014000E401400400FA0582
:1007D0000090D003B40000200148006800470000EA
:1007E0002C00002002E008C8121F08C1002AFAD11C
:1007F00070477047002001E001C1121F002AFBD1A1
:100800007047000072B601F055F900BF00F098FF84
:100810000028FBD1104C0121208801EB00400FA1E2
:1008200001F09AF810480068C00700D000BE208888
:10083000022101EB00400DA101F08EF8BFF34F8FB4
:100840000948E43801680D4A01F4E0611143016090
:10085000BFF34F8F00BFFDE7D000002046617461F9
:100860006C206572726F7200F0ED00E05379737462
:10087000656D207265736574000000000400FA0560
:100880000EB500210091CDE901106A4644F2010045
:10089000FFF7B8FF0EBD00F003B800F009B8000084
:1008A00072B602480168491C016070473C00002094
:1008B00003490868401E086000D162B67047000016
:1008C0003C00002070B5054608680C46411C04D069
:1008D00000F021FE206800F0A9FD6068411C02D0F4
:1008E000002100F091FD2968A069C1F82405607D10
:1008F000227D29681043C1F86C05D4E900122868EC
:10090000C0F81425C0F80C15207D012814D1A0686A
:10091000411C02D0002100F077FDE068411C04D0AA
:1009200000F0F9FDE06800F081FDD4E902122868CA
:10093000C0F80825C0F8101570BD70B505460868E8
:100940000C46411C04D000F0F0FD206800F078FD5A
:100950006068411C02D0002100F05FFD2968A06999
:10096000C1F82405607D217D2A680843C2F86C0522
:10097000D4E900122868C0F80C15C0F81425207DB1
:10098000012814D1A068411C02D0002100F045FDCF
:10099000E068411C04D000F0C8FDE06800F050FDA4
:1009A000D4E902122868C0F80825C0F8101570BDF7
:1009B0002DE9F0470546861C90460F464FF0010989
:1009C0000020FFF768FF1B4C20683860D4E9000165
:1009D000401AA16804F21C47081A0EE001213846AB
:1009E00000F0EEFA00F0E0F90146384600F0E8FACF
:1009F000D4E90001401AA168081A401C8642EDD8CB
:100A0000B8F1000F03D0052065F3891002E006203D
:100A100065F39F50A2682168114004EB8101C86012
:100A20002068304420600020FFF737FF4846BDE8CB
:100A3000F08700008002002030B482680468531CF4
:100A40008360A154D0E901128A4202D330BC00F085
:100A500072BB30BC70470000034803C8814201D11B
:100A600001207047002070478002002005494FF0A8
:100A7000FF32082841F8202002D3084480F84C2097
:100A800070470000D4000020F0B54FF0FF3512B1E0
:100A90000023082601E0082309260C4C05E000BFCE
:100AA00054F823707F1C04D05B1CB342F8D3284653
:100AB000F0BD26185DB286F8245044F82310002AB1
:100AC000F5D1E11881F84C00F1E70000D4000020D6
:100AD0000249084490F9240070470000D400002027
:100AE0002DE9F041154C051E03DD607828B16D1E1F
:100AF00003E002DA607800B16D1C6068104E0127D7
:100B000048B13088626807EB00400EA100F028FF72
:100B10000020FFF7B5FEA068A8420AD03088A3687D
:100B200007EB00402A4614A100F021FF0020FFF748
:100B3000A7FE00206070BDE8F081000000000020EA
:100B4000D00000206D5F61636364626C72656164F4
:100B50002077617320657870656374656420746FB5
:100B600020686176652076616C756520302062753D
:100B700074206973202575006D5F61636372656120
:100B8000642073686F756C64206265202564206240
:100B900075742069732025640000000010B50021E1
:100BA000024800F018FA80F3100010BD9C060020E7
:100BB00010B51E4C6068002806DD607820B16068C2
:100BC000401E60601A4813E06068002807DA607809
:100BD00028B16068401C60601548001D08E0A068EE
:100BE00050B1607840B1A068401EA0601048083045
:100BF0002178405C207001E0002060702078C00700
:100C00004FF01E0002D001F0A3F901E001F040F91D
:100C1000207880074FF01F0003D5BDE8104001F099
:100C200097B9BDE8104001F033B900000C00002076
:100C3000932B00002DE9FC5F0E008346DDE90C4795
:100C4000C6F1000098469246814600D40846012528
:100C500003E000BF90FBFAF06D1C5045FADAA8459E
:100C600000D9454624B1002E01DB780700D5641E6B
:100C7000B80702D5B8F1000F0AD0F80708D13CB187
:100C8000A54205D220215846641EFFF7D5FEF6E79F
:100C9000002E02DA4E462D2102E0780703D52B21E3
:100CA0005846FFF7C9FE07F0030002280BD1B8F140
:100CB000000F08D13CB1A54205D230215846641E30
:100CC000FFF7BAFEF6E7CDE9004743465246314604
:100CD000584601F0F7FEBDE8FC9F000070B50D46D8
:100CE000044600684FF4887100F0D3FF4FF4907110
:100CF000206800F0CEFF4FF49271206800F0C9FF29
:100D00004FF4A271206800F0C4FF20681249C0F8B7
:100D1000041320686907000B40B2090E002806DAA8
:100D200000F00F0000F1E02080F8141D03E000F156
:100D3000E02080F8001420680121000B40B200F090
:100D40001F0291404009800000F1E020C0F88012AD
:100D5000C0F8001170BD0000100302000246002020
:100D60001268930702D0530702D47047500714D576
:100D700002F00300012802D002280CD105E0C2F3E2
:100D800083100B68801C184404E00223086803EBFE
:100D900092521044086001207047086800EB92539B
:100DA000C2F38910401CEEE72DE9FF4100262348DD
:100DB00000F003F92148001F074600F0FEF8204C20
:100DC00060680090A56800E000986946284004EB40
:100DD00080000C30FFF7C2FF0028F5D101AA00996E
:100DE00001EA050304EB8303491CDB6842F8203069
:100DF000401C00910228F2D3019800F00300012862
:100E00000BD0022810D10198032101EB90500099DA
:100E1000BDF80A6001EB900005E00198BDF80A609A
:100E2000C0F3831008440090384600F0C3F808B1BE
:100E30000098606004B03046BDE8F081980600205C
:100E40008002002002240125A103002000F0EEFD15
:100E500008B1FFF715FD00F065FC2049204801F0BE
:100E6000C3F808B1FFF70CFD1E484FF00A080068F0
:100E7000C0B201F0D1FB1C4F0321388801EB0040C8
:100E80001AA100F069FD1F4E4FF0000BB9464FF05C
:100E9000050A00BF05FB04F7384601F0E7FB01F047
:100EA00093F800E020BF30780028FBD0B9F800109C
:100EB0000AEB014014A100F04FFD86F800B038465F
:100EC000FFF70EFE641C4445E4D90124D5F100056A
:100ED00000F036FC0028FBD1DCE70000F92500001B
:100EE000782B000004250140D000002051444543E8
:100EF0002074657374696E672073746172746564BD
:100F00002E000000000000202A0000002DE9F0471C
:100F1000C7880446181D16468946B0FBF7F1B0FB9A
:100F2000F7F207FB12009A193A44D21CB2FBF7F20F
:100F3000DDF820A001E02468491E0029FBD13D1AFC
:100F40008846B54216D818E0BAF1000F05D021182E
:100F500009EB08002A46091D04E0204409EB0801BA
:100F60002A46001DFFF7DEF900202468761BA844FE
:100F7000B74201D9354600E03D46002EE4D1BDE838
:100F8000F087000030B5024659B100F07BFD00212A
:100F9000074C09E004EB810315685B88AB4202D182
:100FA0001160002030BD491C8142F3D3052030BDC3
:100FB000B8000020002100F009B8012100F010B8AD
:100FC00008B56A46FFF759F9009808BD08B56A46A2
:100FD000FFF739F908BD08B56A46FFF71BF908BDE8
:100FE00008B56A46FFF722F9009808BD08B56A46B9
:100FF000FFF750F9009808BD70B504460025284653
:10100000FFF749FC21686268086890420ED9401ECB
:1010100008600178A38AE26801FB0325227A21682F
:10102000101AC0B20A79824200D208710020FFF77C
:1010300034FC284670BD70B505460C460020FFF70D
:101040002AFCE868A98A201AB0FBF1F12A68106826
:10105000431C13600170BDE870400020FFF71DBC09
:1010600010B530B1017A42680368891AC9B21A60B2
:1010700006E00E2010BD03681A68541C1C60117035
:10108000491EC9B2F7D2006800210171084610BD9F
:10109000C20800F007030120895C984008407047AF
:1010A00010B5C20800F00703885C01249C4020436F
:1010B000885410BDF0B505460478154889B0164629
:1010C00040F82420124A08690832A2F10C0742F8BD
:1010D0002400487F385520226846FFF723F90494FE
:1010E0002878385C48B10EB10A4A00E0002269460F
:1010F000281D01F00FF909B0F0BD0EB1064A00E05D
:101100000022694605F10C0000F0D6FFF3E700006D
:101110001C000020A1290000ED2700000FB408B535
:101120000399002904D004AA00926A4600F00FF83F
:1011300001B05DF814FB10B582680446002A05D0A2
:10114000D4E90403216898470020A06010BD2DE970
:10115000FC4791460C00804676D014F8011B39B14B
:1011600025290ED04046FFF767FC20780028F4D1EF
:1011700098F80C00002867D04046BDE8FC47FFF710
:10118000DABF0020012221782B291BD02D2902D083
:10119000302908D102E040F0010001E040F00200F7
:1011A000641C002AEFD100252A290ED02178A1F154
:1011B00030020A2A11D205EB850201EB4205641CBC
:1011C000303DF1E740F00400EAE7D9F800100B1DCC
:1011D000C9F800300968641C0D44217800232E29C9
:1011E0000BD114F8011FA1F130020A2A05D203EB3A
:1011F000830201EB4203303BF3E76C290DD06829F1
:101200000BD0692921D00BDC252918D0582931D0E1
:1012100063290ED0642915D117E014F8011FECE7FB
:10122000702969D0732932D075291BD0782909D14A
:1012300020E0D9F80000011DC9F8001001784046EF
:10124000FFF7FAFB641C90E76CE0D9F800100A1D68
:10125000C9F800200968CDE900500A224046FFF78E
:10126000E9FCEFE7D9F800100A1DC9F80020096869
:101270000A2206E0D9F800100A1DC9F80020096802
:101280001022CDE90050404601F01CFCDAE7D9F805
:10129000001000270A1DC9F800200E68C00705D1FC
:1012A00012E04046761C7F1CFFF7C6FB3178002910
:1012B000F7D104E0202140466D1EFFF7BDFBBD4283
:1012C000C0D9002DF6D1BDE74EB13046FFF74EF83C
:1012D000074604E0202140466D1EFFF7ADFBBD42EE
:1012E00006D9002DF6D103E04046761CFFF7A4FB9B
:1012F00031780029F8D1A5E7D9F80000011DC9F817
:101300000010056830214046FFF796FB78214046E3
:10131000FFF792FB08200021CDE9000103461022CF
:101320002946B0E7BDE8FC872DE9FF411C46DDE911
:101330000A7815460E46684600F0AEF846EA4501C2
:1013400041EA840141EA072242EA0841009A00EB9F
:101350008200C0F80017BDE8FF812DE9FF411C465F
:10136000DDE90A7815460E46684600F0A3F846EA1D
:10137000450141EA840141EA072242EA0841009A14
:1013800000EB8200C0F80017BDE8FF812DE9FF41A6
:101390001C46DDE90A7815460E46684600F098F8C6
:1013A00046EA450141EA840141EA072242EA08414E
:1013B000009A00EB8200C0F80017BDE8FF811CB561
:1013C000002100910B4601220191FFF7C6FF1CBDD1
:1013D0001CB5002100910B4601220191FFF7D6FFB9
:1013E0001CBD0000202802D24FF0A04202E0054AB6
:1013F00000F01F00002302EB800043EA8101C0F8E7
:1014000000177047000300501CB500220B460092E5
:1014100011460192FFF7A1FF1CBD1CB500220B462F
:10142000009211460192FFF7B1FF1CBD1CB50021CF
:1014300000910B46012201911146FFF78EFF1CBD62
:101440001CB5002100910B46012201911146FFF7C6
:101450009DFF1CBD13B50C46684600F01DF80099B1
:1014600000EB8101D1F8002722F44032C1F80027B7
:10147000009900EB8100D0F8001741EA0441C0F860
:1014800000171CBD01B5684600F006F8009A01215E
:101490009140C0F80C1508BD0168202902D24FF018
:1014A000A040704701F01F01016001487047000033
:1014B000000300500168202902D24FF0A04070477D
:1014C00001F01F0101600148704700000003005057
:1014D0000168202902D24FF0A040704701F01F019F
:1014E00001600148704700000003005001B56846E4
:1014F000FFF7D2FFD0F810050099C84000F00100B6
:1015000008BD01B56846FFF7C7FF009A0121914069
:10151000C0F8081508BD01B56846FFF7CBFF009A73
:1015200001219140C0F8081508BD01B56846FFF7D4
:10153000CFFF009A01219140C0F8081508BD0000B6
:101540001CB5094C0144D4E90034CDE900346C46A3
:1015500006E000BF54F82030D3F81035401C08C214
:101560008142F7D81CBD0000A02B0000034908B53C
:101570000844002101600068009008BD0060004040
:1015800002494058012800D0002070470060004008
:1015900030B5124B01460020D3F81044224609E032
:1015A000157A854205D1401C0A28F7DB4FF0FF3041
:1015B00030BD5268002AF3D1421CF9D00872D3F82A
:1015C00010242AB152684A60D3F81024516030BD0B
:1015D0000022C3F810144A6030BD000080020020D1
:1015E000F0B595B01C4615460F4608461A9E00F009
:1015F00019FB182109A8FEF7AEFE0E96CDE9095495
:101600000023082203A9384600F021FB0598069024
:10161000BDF81000ADF81C00BDF81200ADF81E00BA
:1016200000208DF821000398082600F0030001280F
:1016300002D0022818D032E003983346850AC0F35E
:10164000C2008DF8200003980FA9C0F38314A200F4
:10165000384600F0FCFA09A8009006AB22460FA914
:10166000284600F03BFA1AE00398840DC0F3C2004C
:101670008DF82000082C01D2254600E008253346CD
:101680002A460FA9384600F0E2FA2E44641B09AB43
:1016900006AA29460FA800F073F9002CEAD13846B3
:1016A00000F0C6FA15B0F0BD7047012001F0BCB8DB
:1016B000084810B50178084A515C19B1001D00F0C6
:1016C000B5FE02E00C3000F0C3FDBDE81040002084
:1016D00001F0AAB8440000201800002008B5034A11
:1016E00000924023024AFFF77BFF08BDE526000079
:1016F000800100200A4A012902EBC00007D002291C
:1017000007D0032907D0042907D000207047022002
:101710007047042070470079704740797047000097
:10172000382D000010B5FFF7C0FF04210348FFF774
:101730002FFF02490120487210BD00005800002010
:101740002DE9F0478CB0FFF787F918B100200CB0F5
:10175000BDE8F087784C0020C4F81804BFF34F8F21
:1017600060680290A5684FF00008284004EB8000F4
:1017700008E021680298814201D86160E6E72840CC
:1017800004EB80000C3002A9FFF7E8FA0028F0D142
:1017900003AB029901EA050204EB8202491CD268FC
:1017A00043F82020401C02910228F2D3039800F055
:1017B0000300022802D001284ED0A5E00398502251
:1017C000810D8946B2EB905F00D850210E4666F33A
:1017D0009F5003900831594800F0DBF9070078D09A
:1017E00000F020FA4346082203A9384600F035FAF3
:1017F000029908F1080A2940681A8000001D8642F3
:1018000023D94D4D0C3530B1C2B204EB8101301AF1
:1018100090460C3104E02946F2B200259046284655
:10182000C6B25346384600F018FA0AEB08032DB149
:10183000324629464FEA070000F00FFA029909F1F3
:10184000030001EB900002903AE004EB8101534663
:10185000324638460C31EFE70398C0F3831106296E
:1018600000D3062161F389100390C0F38310801C1C
:101870008100324800F08DF9070045D000F0D2F920
:101880004346082203A9384600F0E7F908F10808A2
:1018900000260FE00298434600EA0501401C04EBD5
:1018A00081010290042238460C3100F0D6F908F18B
:1018B0000408761C0398C0F38310B042EAD847B1FD
:1018C000D4F81054D4F8180468B1384600F0B0F9D0
:1018D0002CE019E0687A012804D12A6828463946A4
:1018E000126890476D68002DF4D1384600F0A0F9D9
:1018F0000020FEF7D0FFD4F8180408B90298606001
:101900000020FEF7CAFF11E0D4F8104404E021687B
:101910002046896888476468002CF8D1084802216D
:10192000008801EB004007A100F016F8FFF794F8DB
:1019300080F001000BE7000080020020702D000005
:10194000D00000204261636B656E647320666C7525
:10195000736865640000000000231A4600F0E2BED0
:1019600008B5012300926A4600F0DCFE08BD1CB5F4
:10197000CDE9002302236A4600F0D4FE1CBD00001E
:101980002DE9F0470E4680461C46924608293ED86F
:1019900094F80C90002020731946104600F0D4FDF6
:1019A0000025B54206D218F805201AA12046FFF7F7
:1019B000B5FB03E019A12046FFF7B0FB6D1C082D15
:1019C000EFD317A12046FFF7A9FB0025B54210D29F
:1019D00018F80570FEF7A2FC0068C05D10F03E0F1D
:1019E00001D03A4600E02E220EA12046FFF796FBDA
:1019F00003E00DA12046FFF791FB6D1C082DE5D3F8
:101A000001222146504600F081FD84F80C90BDE88B
:101A1000F0870000202530327800000020202000D0
:101A20007C0000002563000020000000104810B575
:101A3000FF218160002101604160C0F81814C0F8E6
:101A4000141480F820140B4800F0F0F800280DD191
:101A500009480A490A4B401AC108002003E000BFA8
:101A600023F82000401C8842FAD3002010BD00005B
:101A700080020020702D0000702D0000382D000025
:101A8000B800002002480349401AC008704700000F
:101A9000702D0000382D000013B56846FFF772FA6C
:101AA00008B100201CBD0248009950F831001CBD4F
:101AB000382D000070B508480125D0F8104480F892
:101AC000205405E0657221682046496888476468AB
:101AD000002CF7D170BD0000800200202DE9FF47E7
:101AE00081460C9D00200C462F7B28739846164695
:101AF0002946184600F028FD072E42D2DFE806F0FE
:101B000004090F161F2A360049462846FFF706FB30
:101B100037E0494628462268FFF700FB31E0D4E968
:101B2000002349462846FFF7F9FA2AE0A06800900A
:101B3000D4E9002349462846FFF7F0FA21E0D4E92A
:101B40000201CDE90001D4E9002349462846FFF708
:101B5000E5FA16E004F1080007C88DE80700D4E9AB
:101B6000002349462846FFF7D9FA0AE004F10800A5
:101B70000FC88DE80F00D4E9002349462846FFF737
:101B8000CDFA00222946404600F0C0FC2F73BDE884
:101B9000FF872DE9F041858A80462D1F4819C01C1A
:101BA000B0FBF5F0C6B24046FFF726FA041E19D086
:101BB0000020207101206071E58000272546761EF7
:101BC000C4F800800BE04046FFF716FA60B1617977
:101BD000491C6171286005467F1CC0F80080B7422F
:101BE000F1D32046BDE8F081204600F002F8002045
:101BF000F8E72DE9F041457901466B1E002201E02E
:101C00000968521C9A42FBD30F680146002605E082
:101C100038460C68FFF70FFA2146761CAE42F7D320
:101C2000BDE8F0810121001DFFF7CAB9FFF718BA1E
:101C300010B504460121001DFFF7D8F910F0FF0F81
:101C400004D12046BDE81040FFF7D3BF10BD38B522
:101C500001240094FFF75AF938BD38B500240094E8
:101C6000FFF754F938BD4058002800D001207047D4
:101C700008B5002242504058009008BDD0F8040337
:101C8000084000D0012070474058002800D00120B3
:101C9000704708B5002242504058009008BD00002F
:101CA0002DE9F0410E46804600F018FC204D00283A
:101CB000404616D0FEF70CFF284490F84C008009EF
:101CC000032802D001280AD003E04046FFF70EFCAB
:101CD00028B103214046BDE8F041FFF7BBBB02211C
:101CE000F8E700F007FC002820D04046FEF7F0FEA1
:101CF0000446104F4FF4807007EB840100EB840022
:101D0000D1F8102580B242F00102C1F81025FFF78A
:101D10002DFC002E0AD04046FEF7DAFE55F82000D2
:101D2000002803D00120A040C7F80403BDE8F081DB
:101D3000D4000020006000402DE9FC41DFF8C080A5
:101D4000044608EB0400002790F924001346C0174E
:101D50000E46401C01D008274FE0B0781946C0F36A
:101D600040022046FEF790FE0546401C44D0B07865
:101D700041071CD4C0070DD068460094FFF78CFBC8
:101D8000009900EB8100D0F8001721F00201C0F8A3
:101D9000001707E000217378204600910A46019160
:101DA000FFF7C2FA164920465531FFF779F9B078A6
:101DB000800718D51348317800EB8500D0F810253E
:101DC000114B1A40C0F810254FF47C524FF44033A9
:101DD00002EA042203EA01410A43D0F810150A433B
:101DE000C0F8102509E008EB0500327810F84C1F08
:101DF00041EA8211017000E004273846BDE8FC8109
:101E0000D400002000600040FFC0FCFF70B5184DFA
:101E100095F85B0008B1082070BD0020411E2A180B
:101E2000401CC0B282F824103028F8D30024204689
:101E3000FEF71CFE641CE4B2092CF8D3002445F81C
:101E4000554F0C49AC80E02081F800040126402069
:101E5000891FC1F88002C1F800014FF4BE70FFF77E
:101E600085FB0549F007C1F80403AE71204670BD3B
:101E7000D400002006E000E000600040034890F835
:101E80005B00002800D0012070470000D400002033
:101E9000FFF7F8BA2DE9FC4104462A480D462044D4
:101EA000002690F92410491C01D0082643E0A978A7
:101EB000002751B3012200212046FEF7E5FD411C19
:101EC00021D0830020482A7818446978D0F810354A
:101ED000DFF878C003EA0C03C0F81035D0F81035ED
:101EE0004FF47C5C0CEA042C43EA0C034FF4403CB6
:101EF0000CEA02424FF4801C0CEA01510A431343DE
:101F0000C0F8103504E0042615E0FE2180F8241006
:101F100068780128204611D0FFF7B4FA0122204644
:101F20000097002311460197FFF7FEF90549204667
:101F30005531FFF7B5F83046BDE8FC81FFF7E1FA0F
:101F4000ECE70000D400002000600040FFC0ECFF80
:101F5000FFF7D7BA0121B1EB507F01D101207047C3
:101F60000020704770B50D4600F03AFB04000FD01A
:101F70000020FEF790FC207920B10020FEF78DFCB8
:101F8000112070BD0120256020710020FEF785FC26
:101F9000002070BD10B500F023FB002802D0002106
:101FA0000160017110BD0000044901200860044A6D
:101FB00000211160034908707047000004200140AF
:101FC0000025014034000020044901200860044934
:101FD0000860044902200870704700000025014095
:101FE000002001403400002070B52B4D04462878B5
:101FF00008B1082070BD6960284960780860002138
:10200000E068FFF7EFF900216068FFF7EBF90021C6
:10201000A068FFF7E7F9214BD4E901211833E06804
:102020001A601A1D1160191F08601C492069383197
:1020300008601A49207D091F0860194AD2F8000279
:1020400040F00100C2F800021448617D20300123F5
:10205000002609B1036000E0066021780420082909
:1020600003D00E48083001600620A17D09B140F080
:102070000100C2F80403E07D0A49400181F8000430
:102080004FF0E0224FF480213046C2F88012C2F8AF
:1020900000112B7070BD00003400002008250140A5
:1020A0000020014012E000E00149024800F0E4BBDA
:1020B00030010020002000402DE9F0410546007964
:1020C00016460F4600EB40012D4A01EBC00102EB22
:1020D000810494F82A1011B10820BDE8F081294943
:1020E00051F820102868FFF73DFF08B11120F4E7F0
:1020F00039462846FEF7E6FB666038692060300006
:102100004FF001062FD03F7F4FF48E712868FFF704
:10211000AFFD4FF4A2712868FFF7AAFD28681A499D
:10212000C0F8041328684FEA4711000B40B200289A
:1021300006DA00F00F0000F1E02080F8141D03E043
:1021400000F1E02080F800142868000B40B200F095
:102150001F0206FA02F14009800000F1E020C0F8F9
:102160008012C0F8001128680421C0F80015002072
:10217000A061E06184F8290044F8140FA675ACE76B
:1021800030010020A82B0000800002002DE9F0475C
:10219000054600790B4600EB400101EBC0002349E6
:1021A00001EB8004284600F043F810B11120BDE88F
:1021B000F0874FF00008C4F82080A360626184F8C3
:1021C00028804FF48E76474631462868FFF750FD49
:1021D00028684FF00109C0F808902146286800F0EF
:1021E000E7FA606800BBD5F800A00EE094F828007C
:1021F00008B10F2716E031465046FFF734FD00289E
:10220000F4D02146504600F0D3FA216A6069814239
:10221000F1D331462868FFF726FD0028F9D0286859
:10222000C0F80C90C4F814803846C0E73001002094
:10223000007900EB400101EBC000044901EB800094
:102240004069002800D001207047000030010020C4
:102250002DE9F047044600794FF0000900EB4001FA
:1022600001EBC000254901EB80072068C0F800950C
:10227000786880B120682249C0F8081320680121DD
:10228000000B40B200F01F0291404009800000F1B5
:10229000E020C0F880112068D0F80C25D0F8148513
:1022A000D0F80865D0F810554FF0FF31C0F814157C
:1022B000C0F80C152068C0F80815C0F81015501C9F
:1022C00002D01046FFF77BF8B8F1FF3F02D040463E
:1022D000FFF775F8681C02D02846FFF770F8701CED
:1022E00002D03046FFF76BF82068FFF753FE87F8FF
:1022F0002A90C7F80490BDE8F08700003001002064
:10230000840202000149024800F062BB5C01002027
:10231000002000402DE9F0410546164600790F46A1
:10232000154A00EBC00102EB810494F8201011B1B2
:102330000820BDE8F081114951F820102868FFF706
:1023400011FE08B11120F4E739462846FEF7F5FAE8
:102350006660386920601EB1397F2846FEF7BEFCF2
:1023600028680821C0F800150020A061E061012163
:10237000606184F82010DCE75C010020AC2B0000D9
:102380002DE9F04704460E460079204900EBC000D5
:1023900001EB800517463046FFF7DCFD30B12046E3
:1023A00000F036F820B11120BDE8F0871020FBE7DF
:1023B0006F61AE604FF49076002731462068FFF7DA
:1023C00068FC4FF4AC7841462068FFF762FC206857
:1023D000AA686969C0F84425C0F848152068012139
:1023E0008160686878B9B14649462068FFF74CFCBF
:1023F000064641462068FFF747FC0643F4D000B18B
:102400000F27002068613846CEE700005C010020FD
:102410000079054900EBC00001EB8000406900280D
:1024200000D00120704700005C0100202DE9F0473A
:1024300004460079274900EBC00001EB80072068C3
:102440004FF00009C0F80095786880B120682249F3
:10245000C0F8081320680121000B40B200F01F02F1
:1024600091404009800000F1E020C0F88011206810
:10247000D0F80C25D0F81485D0F80865D0F81055A0
:102480004FF0FF31C0F80C15C0F814152068C0F8E3
:102490000815C0F81015501C02D01046FEF798FF22
:1024A000B8F1FF3F02D04046FEF792FF681C02D011
:1024B0002846FEF78DFF701C02D03046FEF788FFDD
:1024C0002068FFF767FD87F82090C7F80490BDE803
:1024D000F08700005C01002010030200044908445A
:1024E00090F92400082801DB012070470020704784
:1024F000D40000200449084490F92400082801D29F
:102500000120704700207047D400002010B50C4611
:10251000017A052908D0407A38B1084808A1026834
:102520002046FEF7FBFD00E01AB106A12046FEF7AB
:10253000F5FD2046BDE81040FEF7FDBD90000020EF
:10254000257300000D0A000038B5C3880D46044607
:1025500033B114A0009015A216A12846FEF7DEFDA7
:10256000217A05291CD0607A48B1A088FFF7C2F80B
:10257000164951F8202016A12846FEF7CFFDA08865
:102580000021FFF789FA03461049207A143951F8DF
:10259000202001B02846BDE830400EA1FEF7BEBDA8
:1025A00038BD00001B5B306D000000001B5B313B41
:1025B00033316D0025734C6F67732064726F7070D8
:1025C0006564202825642925730D0A0090000020E9
:1025D000257300003C25733E2025733A200000003F
:1025E0000349884201D1034870470020704700002A
:1025F000002000402C00002082B2B2F5827F08D17A
:102600008AB204494A600014886001200870FFF70C
:10261000CBBC7047000000201CB504461148006880
:1026200000900020019003208DF80100FFF726FCA8
:1026300008B9FFF7EBFB14B902208DF800000A4A35
:1026400069461D20FFF778FB01211D20FFF728FBBD
:1026500001A91F20FFF71EFC01A91E20FFF71AFC8D
:102660001CBD0000902B0000B10B0000002100F009
:1026700001B80000024A506091600120507070471C
:102680000C00002070B5054688690C4600284FF400
:10269000847128460AD0FFF7EBFAD5F81805626A6C
:1026A000E1688854606A401C606270BDFFF7E0FA20
:1026B000D5F8180570BD1FB501238DF80030CDE9A0
:1026C0000121D0E90012684690471FBD1FB50123C4
:1026D0008DF800308DF808100192D0E9001268469C
:1026E00090471FBD70B50D4C0020D2B22070201D48
:1026F0000B4D0378EB5C1BB1001DFFF741FE02E0C0
:102700000C30FFF743FD08B1FEF7BAF860780028F7
:1027100002D021780029FAD070BD000040000020CE
:10272000180000202DE9F84F204D924689460646B4
:102730009846012269461846AF68FEF739F958B342
:10274000009800210446801C09E000BF00EA07034E
:102750005AF8212005EB8303401C491CDA604145EF
:10276000F4D34FEA164AFEF719FA4AEA0041601C10
:10277000384005EB80003C4005EB8402C160D06826
:1027800066F3C50068F3891069F39F2020F0030009
:10279000401C20F00400D06095F8200402E000BF47
:1027A000FEF7CEFF0028FBD1BDE8F88F80020020A5
:1027B00070B50C4605464FF48E71FFF759FA216A41
:1027C000A068415C206A401C2062C5F81C1570BDE1
:1027D0001FB500228DF800200291816801914261AD
:1027E000D0E90012684690471FBD00001FB50A4699
:1027F00001788DF8001041680191017A8DF8081078
:10280000C0680390044850F82210083850F822207D
:10281000684690471FBD00002400002001490120A8
:10282000087070474000002010B588B00446202290
:102830000E496846FDF776FD06200090C01F019006
:10284000029003904FF0EB7006900CB1084A00E044
:10285000002269460748FEF72DFC08B1FEF710F884
:102860000448001F447008B010BD0000CC2B0000CD
:102870001D280000440000202DE9FF470C460546B6
:102880004FF40071FFF7FAF901274FF401780026A1
:1028900018B34FF4927949462846FFF7E4F9E0B1BE
:1028A00049462846FFF7E4F9C5F8088394F829005B
:1028B00000B96F6002208DF80000D5F88004C5F8DB
:1028C00080040390A0690290E0680190A661E6612F
:1028D000D4E900126846904728E004212846FFF713
:1028E000CDF918B34FF484712846FFF7BCF9E8B16D
:1028F00021462846FFF7C6FE616AA069884215D1C5
:10290000E06938B1E268616AA0612069E6616662E7
:10291000E06008E094F8290000B96F60C5F808830A
:10292000A661E268616A2046FFF7C5FE4FF48E7823
:1029300041462846FFF797F978B1206A61698842D5
:1029400002D294F8280020B341462846FFF790F9B8
:10295000616911B12046FFF73BFF4FF4A278414671
:102960002846FFF780F9002818D041462846FFF78F
:102970007FF994F8290000B12F60A06900280DD0DC
:10298000A661E268616A04B02046BDE8F047FFF73F
:1029900092BE21462846FFF70BFFDEE7BDE8FF8722
:1029A0001FB50A4601788DF8001041680191017A3F
:1029B0008DF80810C0680390044850F822100838B9
:1029C00050F82220684690471FBD000024000020D8
:1029D0002DE9FF410C464FF4927705463946FFF743
:1029E00053F90026C0B139462846FFF752F90220B4
:1029F0008DF80000D5F88004C5F880040390D5F860
:102A00003C058DF80800E0680190A661E661D4E914
:102A100000126846904723E04FF4887739462846ED
:102A2000FFF732F9E0B139462846FFF732F9D5F819
:102A30003C15A069884213D1E06960B1E268D5F81D
:102A4000000220F02000C5F80002E069A0612069C2
:102A5000E661E06001E0A661E2682046FFF736FE2D
:102A60004FF4A27739462846FFF70EF960B1394690
:102A70002846FFF70EF9A06930B1A661D5F83C15DC
:102A80002046E268FFF722FE4FF490773946284649
:102A9000FFF7FAF8002813D039462846FFF7F9F86F
:102AA000606900280CD0D5F84C058DF800608DF8D1
:102AB0000800A06801906661D4E90012684690475A
:102AC000BDE8FF812DE9F05F8346DDE90A4A9946BA
:102AD00090460D460846012703E000BFB0FBF8F022
:102AE0007F1C4045FAD2B94500D94F465FEACA700B
:102AF00012D18CB15FEA8A7002D5B9F1000F01D012
:102B0000202607E0302605E031465846641EFDF7D2
:102B100093FF0CB1A742F7D35FF00106B9F1010FA3
:102B200002D9A9F1010903E0B5FBF6F0404502D353
:102B300006FB08F6F2E7DFF83C9000BFB5FBF6F0C5
:102B400000FB165519F800105846FDF775FFB6FB47
:102B5000F8F6002EF2D15FEACA7009D0002C07D037
:102B6000A74205D220215846641EFDF765FFF5E710
:102B7000BDE8F09FB02B000000070000030000003C
:102B8000040000001C0000003200000001000007EB
:102B9000020002010300020200030103020100001F
:102BA0000000005000030050A92000000523000091
:102BB0003031323334353637383941424344454673
:102BC000DD160000B1160000A9160000FFFFFFFF90
:102BD000FFFFFFFFFFFFFFFFFFFFFFFF0000000001
:102BE000000000000000D601070100000040404046
:102BF00040404040404041414141414040404040D0
:102C0000404040404040404040404040400502027B
:102C1000020202020202020202020202022020203A
:102C20002020202020202002020202020202909096
:102C30009090909010101010101010101010101094
:102C400010101010101010100202020202028888E8
:102C500088888888080808080808080808080808F4
:102C600008080808080808080202020240000000DC
:102C7000ED2B00007761726E696E670064656275A6
:102C8000670000001B5B313B33306D001B5B306D18
:102C9000000000001B5B313B33316D001B5B313B9F
:102CA00033326D001B5B313B33336D001B5B313BBB
:102CB00033346D001B5B313B33356D001B5B313BA7
:102CC00033366D001B5B313B33376D00696E666FC9
:102CD000000000006572726F720000004750494F9B
:102CE0005445000050525300514445430000000039
:102CF0005541525400000000554152544500000017
:102D000062616C6C6F632E6C6F675F6D656D706F69
:102D10006F6C000061707000882D000000000020C2
:102D2000D4000000E40700005C2E0000D400002066
:102D3000D4250000F4070000DC2C00000000000097
:102D4000E42C000000000000E82C0000000000005F
:102D5000F02C000000000000F82C00000000000033
:102D6000002D000000000003142D000000000303EC
:102D70006C000020640000206C000020C0010020D6
:102D8000CC0000201800000000010000000000003E
:102D90000000000000000000000000000000000033
:102DA0000000000000000000000000000000000023
:102DB0000000000000000000000000000000000013
:102DC0000000000000000000000000000000000003
:102DD0000020004000000000002000400000000033
:102DE000C02B0000000000000000000000000000F8
:102DF00000000000000000000000000000000000D3
:102E00000000000000000000D42C0000742C000022
:102E1000CC2C00007C2C00008C2C0000842C0000AA
:102E2000942C00009C2C0000A42C0000AC2C000072
:102E3000B42C0000BC2C0000C42C00000090D00377
:102E40000000000000000000000000000000000082
:0C2E500000000000000000000000000076
:0400000500000201F4
:00000001FF
